:100000001AC033C032C031C030C02FC02EC02DC086
:100010002CC02BC02AC029C028C027C042C325C07D
:1000200024C023C022C021C020C01FC00CC3E6C210
:100030001CC01BC0B00411241FBECFEFCDBFDFE337
:10004000DEBF2FE3A0E0BFE301C01D92A734B207DB
:10005000E1F710E0CBE1D0E003C02197FE01A4D688
:10006000CA31D107D1F773D3B1C6CACFAF92BF920D
:10007000CF92DF92EF92FF920F931F93CF93DF9374
:100080006C017B018B01040F151FEB015E01AE18A3
:10009000BF08C017D10759F06991D601ED91FC91C5
:1000A0000190F081E02DC6010995892B79F7C501F2
:1000B000DF91CF911F910F91FF90EF90DF90CF9044
:1000C000BF90AF900895FC01508D418D252F30E0F9
:1000D000842F90E0821B930B541710F00F96089515
:1000E00001970895FC0196898789981761F0A7897F
:1000F000AE0FBF2FB11D5D968C9197899F5F9F704A
:10010000978B90E008958FEF9FEF0895FC019689FB
:100110008789981731F08789E80FF11D858D90E068
:1001200008958FEF9FEF0895FC0196892789892F05
:1001300090E04096821B91098F7099270895CF9384
:10014000DF93EC01E881F9810284F385E02D0995C4
:10015000EC85FD8586818F738683EC85FD858581A1
:100160008F7585838F898E8B1D8ADF91CF9108953E
:100170008F929F92AF92BF92DF92EF92FF920F9376
:100180001F93CF93DF93EC014A015B01E22E8D892F
:10019000882339F0E881F9810088F189E02DCE01CA
:1001A00009950C8910E0FFB6F894EC85FD858681F1
:1001B0008D7F86831D8AD090251160E078E689E8DE
:1001C00099E0A5019401BED5AD2DDD0CBB0BBC5F44
:1001D000E5D57C5F8F4F9F4FEC85FD852BE0959596
:1001E0008795779567952A95D1F760877187EC8514
:1001F000FD85E782EC85FD858681806C8683EC85B4
:10020000FD85858180688583909101028B89809529
:1002100089239801220F331FF901E00FF11FEC0F22
:10022000FD1F9089892B809301028685863028F5F1
:1002300090E0FC01EE51F24740814F3FF1F0FC01AC
:10024000E452F247A08150E2A59FD0011124BC5F87
:100250008A529247FC015081F0E0E0E05F3F29F0D4
:10026000CD014096FC01E50FF11D9FB7F894129661
:100270004C938081886080839FBFF901E00FF11F5C
:10028000EC0FFD1F8785863000F590E0FC01EE51F4
:10029000F24770817F3FC9F0FC01E053F247408193
:1002A000442329F04031B1F1403809F44BC0FC013E
:1002B000E452F247E08140E2E49FF0011124FC5F48
:1002C0004081472309F441C07583020F131FC00FFB
:1002D000D11F8F85863088F490E0FC01EE51F24703
:1002E00020812F3F51F084529247DC01EC91B0E223
:1002F000EB9FF0011124FC5F2183FFBEDF91CF91C2
:100300001F910F91FF90EF90DF90BF90AF909F9063
:100310008F900895FC01EA52F2476081673081F0C6
:10032000633008F06F5FE091010A41E050E001C0E6
:10033000440F6A95EAF740954E234093010AB7CFE0
:1003400060E0F1CF10928006B2CF8A529247DC0172
:100350008C91309761F08F3F51F07096E80FF11D4E
:100360009FB7F8948081886080839FBFAECFF0E014
:10037000E0E0F6CFCF93DF93FC01908D818DA485D3
:10038000B585981309C015968C9115978F7D159694
:100390008C93DF91CF910895C18DCE0FDF2FD11DAA
:1003A0002DA5818D90E001968F709927818F80E433
:1003B00014968C93A485B58512962C93908D818D7F
:1003C0009813E7CFA485B58515968C9115978F7DE9
:1003D00015968C93838D8823E1F2848D809313018D
:1003E000138ED7CFDC011C96ED91FC910FB607FE62
:1003F00003C0258125FD03C0248125FDBBCF0895C1
:10040000EF92FF920F931F93CF93DF93EC0181E064
:100410008D8B988D898D98131CC0AC85BD851496E5
:100420008C91149785FF15C012966C93AC85BD8591
:1004300080E414968C93EC85FD8585818F7D858382
:1004400081E090E0DF91CF911F910F91FF90EF90AD
:1004500008958091110180FF08C0809113018C8F55
:100460008A8D8093130181E08B8FF62E088D10E02A
:100470000F5F1F4F0F701127E02E898D8E1103C063
:10048000CE01B0DFFACFE88DEC0FFD2FF11DF5A600
:10049000088FEC85FD8585818062D1CFCF93DF9376
:1004A000FC0125892223C1F0EC018091110180FF1C
:1004B00008C080911301848F828D8093130181E0A5
:1004C000838FEC85FD85858185FD03C0848186FD54
:1004D00003C0CE0187DFF5CFDF91CF91089581E092
:1004E00008958FB7F8942091063F3091073F4091CF
:1004F000083F5091093F98E09093840A90918E0AAA
:1005000091FFFCCFE091A20AF091A30A90918D0A8D
:1005100090FF08C0BF016627672B21F42E5F3F4F75
:100520004F4F5F4F8FBFBF0176956795CF01860F05
:10053000911DE62FE695E695762F72957F70E71B65
:10054000FF0B67FD3196E80FF91FA0E3B3E01CD461
:100550006E0F7F1F811D911D0895DC01ED91FC91AF
:100560000684F785E02D23E030E00994FC0101903A
:100570000020E9F73197AF01481B590BBC018AE015
:100580009FE374CD8F929F92AF92BF920F931F9370
:10059000CF93DF93CDB7DEB7A197CDBFDEBF19A252
:1005A000423008F44AE08E010F5D1F4F842E912CDB
:1005B000B12CA12CA5019401C5D3E62FB901CA0124
:1005C000EA30D4F4E05DD801EE938D01232B242B87
:1005D000252B81F790E080E0109711F0CD01C6DF68
:1005E000A196CDBFDEBFDF91CF911F910F91BF903C
:1005F000AF909F908F900895E95CE5CF1F920F9286
:100600000FB60F9211242F933F934F935F936F93E5
:100610007F938F939F93AF93BF93EF93FF938AE062
:100620009FE3A8DEFF91EF91BF91AF919F918F91D2
:100630007F916F915F914F913F912F910F900FBEDE
:100640000F901F9018951F920F920FB60F921124C2
:100650002F938F939F93EF93FF93E091163FF09129
:10066000173F818181FD1BC090818091203F8F5F6A
:100670008F702091213F821741F0E091203FF0E000
:10068000E65FF04C958F8093203FFF91EF919F9113
:100690008F912F910F900FBE0F901F901895808112
:1006A000F4CF1F920F920FB60F9211242F933F9306
:1006B0004F935F936F938F939F93AF93BF9380916B
:1006C000023F9091033FA091043FB091053F4091BC
:1006D000003F5091013F9A01205D3C4F283E63E06E
:1006E000360728F0285E33400196A11DB11D2093E6
:1006F000003F3093013F8093023F9093033FA093CC
:10070000043FB093053F8091063F9091073FA09131
:10071000083FB091093F0196A11DB11D8093063F8E
:100720009093073FA093083FB093093F81E08093E7
:100730008D0ABF91AF919F918F916F915F914F9172
:100740003F912F910F900FBE0F901F90189588ED3D
:1007500090E084BF9093610083E5809302068EE071
:100760008093050680E280930306809100068160F5
:100770008093000691E0909302029093030A8EEF1B
:100780008093260A8093270A80E88093280A809322
:100790002A0A80932C0A8093290A80932B0A80933B
:1007A0002D0A2BE02093000A2DEF31E02093AE0AB2
:1007B0003093AF0A90938C0A1092810A8093820A38
:1007C00081E18093800A789490931E3F40E052EC40
:1007D00061E070E08AE09FE3C0DEC7E0D1E0C09353
:1007E0000606D093080680910B0680FFFCCF60912F
:1007F000100670911106072E000C880B990B7BD107
:100800002DE038E643E55BE32BD26B017C014B0125
:100810005C01AC019B0191D2882319F182E09EE832
:10082000A5DE80E19EE8A2DE5CDE6B017C0128EEA5
:10083000C20E23E0D21EE11CF11C88EEC81683E034
:10084000D806E104F10430F44CDEC616D706E806FB
:10085000F906D0F346DE6C157D058E059F05D0F3B5
:10086000BECF26013701E89477F82FEF3FEF4FE72F
:100870005FE7C301B20161D281110CC02FEF3FEFDE
:100880004FE75FE7C301B20100D118161CF486E000
:100890009EE8C6CF2FEF3FEF4FE75FE4C701B601F9
:1008A000DAD118161CF48AE09EE8BACF2FEF3FEF9A
:1008B0004FE75FECC701B601E8D087FDF4CF20E039
:1008C00030E0A901C701B601E0D087FF0AC06DE2A0
:1008D0008AE09FE395DD46015701B7FAB094B7F877
:1008E000B0942AE037ED43EA5BE3C501B40161D07F
:1008F0004B015C01CFD06B017C01FBD09B01AC01B3
:10090000C501B40155D04B015C014AE0C701B601F5
:1009100039DE8EE09EE82ADE20E030E040E251E45D
:10092000C501B4019DD14B015C01B4D06B01F12C28
:10093000E12C4AE0C701B60125DEC701B601D9D0D6
:100940009B01AC01C501B40133D020E030E040E2AE
:1009500051E486D19FD090E080E04AE013DE61CF81
:10096000EAE0FFE31282138288EE93E0A0E0B0E0B9
:1009700084839583A683B7838CEE9DE880839183DF
:1009800080E098E08487958781E086871786108AC3
:1009900093E0918B92E0928B838B148A158A168A4E
:1009A000178A108E118E87E1828F138E148E089510
:1009B0005058BB27AA270E94F0040C94F1050E940E
:1009C000E30538F00E94EA0520F039F49F3F19F45E
:1009D00026F40C94E0050EF4E095E7FB0C94DA05A0
:1009E000E92F0E94020658F3BA17620773078407BB
:1009F000950720F079F4A6F50C9424060EF4E09502
:100A00000B2EBA2FA02D0B01B90190010C01CA01C8
:100A1000A0011124FF27591B99F0593F50F4503E73
:100A200068F11A16F040A22F232F342F4427585F65
:100A3000F3CF469537952795A795F0405395C9F77D
:100A40007EF41F16BA0B620B730B840BBAF0915035
:100A5000A1F0FF0FBB1F661F771F881FC2F70EC0D4
:100A6000BA0F621F731F841F48F4879577956795A7
:100A7000B795F7959E3F08F0B0CF9395880F08F093
:100A80009927EE0F9795879508950E94B60508F46B
:100A900081E008950E940A0688F09F5798F0B92FC8
:100AA0009927B751B0F0E1F0660F771F881F991FA3
:100AB0001AF0BA95C9F714C0B13091F00E9424061B
:100AC000B1E008950C942406672F782F8827B85F2B
:100AD00039F0B93FCCF3869577956795B395D9F7FB
:100AE0003EF490958095709561957F4F8F4F9F4F05
:100AF0000895E89409C097FB3EF490958095709511
:100B000061957F4F8F4F9F4F9923A9F0F92F96E959
:100B1000BB279395F695879577956795B795F111CE
:100B2000F8CFFAF4BB0F11F460FF1BC06F5F7F4F6B
:100B30008F4F9F4F16C0882311F096E911C077237D
:100B400021F09EE8872F762F05C0662371F096E886
:100B5000862F70E060E02AF09A95660F771F881F55
:100B6000DAF7880F9695879597F90895990F0008F9
:100B7000550FAA0BE0E8FEEF16161706E807F9076F
:100B8000C0F012161306E407F50798F0621B730B0A
:100B9000840B950B39F40A2661F0232B242B252B8B
:100BA00021F408950A2609F4A140A6958FEF811D2E
:100BB000811D089597F99F6780E870E060E00895CF
:100BC0009FEF80EC089500240A9416161706180665
:100BD0000906089500240A94121613061406050641
:100BE0000895092E0394000C11F4882352F0BB0FD2
:100BF00040F4BF2B11F460FF04C06F5F7F4F8F4F35
:100C00009F4F089557FD9058440F551F59F05F3F6F
:100C100071F04795880F97FB991F61F09F3F79F01E
:100C200087950895121613061406551FF2CF4695A0
:100C3000F1DF08C0161617061806991FF1CF869522
:100C40007105610508940895E894BB276627772706
:100C5000CB0197F908950E94B60508F48FEF089527
:100C60000E9443060C94F1050E94E30538F00E94AF
:100C7000EA0520F0952311F00C94DA050C94E005B8
:100C800011240C9425060E94020670F3959FC1F36F
:100C9000950F50E0551F629FF001729FBB27F00D2A
:100CA000B11D639FAA27F00DB11DAA1F649F66277F
:100CB000B00DA11D661F829F2227B00DA11D621FCE
:100CC000739FB00DA11D621F839FA00D611D221F88
:100CD000749F3327A00D611D231F849F600D211D6C
:100CE000822F762F6A2F11249F5750409AF0F1F0EF
:100CF00088234AF0EE0FFF1FBB1F661F771F881F58
:100D000091505040A9F79E3F510580F00C94DA05B0
:100D10000C9425065F3FE4F3983ED4F386957795CF
:100D20006795B795F795E7959F5FC1F7FE2B880FFD
:100D3000911D9695879597F908950E94B605880BA1
:100D4000990B0895A1E21A2EAA1BBB1BFD010DC031
:100D5000AA1FBB1FEE1FFF1FA217B307E407F5076B
:100D600020F0A21BB30BE40BF50B661F771F881F47
:100D7000991F1A9469F760957095809590959B01DD
:100D8000AC01BD01CF01089515D0A59F900DB49F72
:100D9000900DA49F800D911D11240895B7FFF4CFED
:100DA000F3DF821B930B0895EE0FFF1F0590F49164
:100DB000E02D0994A29FB001B39FC001A39F01D071
:100DC000B29F700D811D1124911D0895F894FFCFDD
:100DD0008010101010000607010203000000000040
:100DE00000004080020408010000000000023600FC
:100DF0009400720086004E02AD02B8009F006F02A0
:100E000063006E616E00696E66006F7666002E008C
:030E10000D0A00C8
:00000001FF
